:020000021000EC
:10F8000011241FBE1CC0CF93DF93AC0120E030E079
:10F810002817390760F4A0EDB7E0C0E0D0E0CD01D3
:10F820000197F1F72F5F3F4F24173507C0F3DF91A2
:10F83000CF9108958CB95E9BFECF5E9A0895CCED72
:10F84000DFE0DEBFCDBFCC24DD247601C25EDE4F1B
:10F85000C882D982EA82FB82CE51D140CE5DDE4F92
:10F8600019821882C252D1403324032D6624772492
:10F8700046015701230180916400846080936400F5
:10F8800080916500846080936500599A80E189B910
:10F8900088E18AB900005F9920C041145104E9F45D
:10F8A00024E030E040E050E0C9010197F1F708940E
:10F8B000811C911CA11CB11C11EE811617E691064A
:10F8C00015E3A10610E0B10618F041E0442E512CDA
:10F8D0005F9903C04114510439F30894411C511C31
:10F8E00041145104C1F221E04216510409F081C2D1
:10F8F00020E031E04316510421F4442455241CB186
:10F9000004C05F9BFECF8CB1182F822F99278330C4
:10F91000910551F1843091054CF481309105B1F09D
:10F9200082309105DCF4892B59F050C08530910567
:10F9300071F185309105FCF0069709F444C046C08A
:10F940001B3109F043C021E0012FD3CF113011F05A
:10F95000131571F6312E22E00127CBCF812F992785
:10F96000782E662423E005C0812F9927682A792AFA
:10F9700024E00127BECF1E3009F0BACF25E00127D1
:10F98000CE5DDE4F19821882C252D140B2CFCE5D19
:10F99000DE4FE881F981C252D140EC0FFD1F118387
:10F9A000CE5DDE4F88819981C252D1400196CE5DF5
:10F9B000DE4F99838883C252D1400127861597056F
:10F9C00029F426E096CF101721F092CF273009F0C6
:10F9D00090CFE9818E2F99278331910509F40EC1CB
:10F9E00084319105F4F48630910509F4DBC0873049
:10F9F00091057CF48230910509F483C1833091052F
:10FA000024F4019709F448C0C1C1039709F45BC00D
:10FA1000BDC1803191050CF4B9C142970CF471C19C
:10FA2000B8C08831910509F480C08931910564F42A
:10FA30008531910509F4E2C0853191050CF466C168
:10FA4000469709F463C1A2C18A31910509F462C0E5
:10FA50008A3191050CF48AC08B31910509F44FC0AD
:10FA60004D9709F093C19D81903359F48F8188237C
:10FA700011F48EE107C0813011F487E903C082E000
:10FA800001C080E017E0612E712C1A821B829C83DA
:10FA90001D828E831F827FC1BBE06B2E712C1A8268
:10FAA00088E08B8381E48C8386E58D8382E58E8379
:10FAB00089E48F8383E5888780E589878FE58A8756
:10FAC00082E38B8768C18A8199278039910551F03B
:10FAD000813991056CF08139910531F082399105B8
:10FAE00029F006C08FE005C082E003C08AE001C0B3
:10FAF00080E0A3E06A2E712C1A828B834CC18D8129
:10FB0000882311F48EE12BC0813011F487E927C0DE
:10FB100082E025C0F4E06F2E712C1A8289E0E1E0CA
:10FB2000F0E08093680084911EC08B81803589F459
:10FB30008C81883039F489E0E2E0F0E0809368005D
:10FB400084910DC089E0E0E0F0E08093680084914A
:10FB500006C089E0E3E0F0E0809368008491E4E08F
:10FB60006E2E712C1A828B831C8215C18D81836C41
:10FB700099E0E1E0F0E0082E90936800E89580912C
:10FB8000680080FDFCCF73E0672E712C1A821B8207
:10FB900002C1C25EDE4F188219821A821B82CE51C8
:10FBA000D140AFC08A819927AA27BB27F82EEE241F
:10FBB000DD24CC248B819927AA27BB27DC01992738
:10FBC0008827C82AD92AEA2AFB2A8C819927AA27BA
:10FBD000BB27BA2FA92F982F8827C82AD92AEA2A03
:10FBE000FB2A8D819927AA27BB27C82AD92AEA2A66
:10FBF000FB2ACC0CDD1CEE1CFF1C83C08A819927DC
:10FC0000582F44278B819927482B592BBE01655FBC
:10FC10007F4F46015701E33109F05DC0C25EDE4F00
:10FC2000088119812A813B81CE51D140003088EF73
:10FC3000180781E0280780E03807F8F483E0F8012E
:10FC400020935B0080936800E8958091680080FDB8
:10FC5000FCCFC25EDE4F088119812A813B81CE51E3
:10FC6000D14000501F4F2F4F3F4FC25EDE4F0883E1
:10FC700019832A833B83CE51D140A1E0FB0121911E
:10FC80008191BF019927982F88273327822B932BA7
:10FC90000C01F601E0925B00A0936800E895112446
:10FCA00002E010E020E030E0C00ED11EE21EF31EA4
:10FCB0004250504019F785E0F401A0925B00809318
:10FCC0006800E8958091680080FDFCCF81E1809319
:10FCD0006800E89516C0CEBABB27AF2D9E2D8D2D9E
:10FCE0008FBB0894C11CD11CE11CF11CDB018D9160
:10FCF000BD018DBBE29AE19AE199FECF415050409F
:10FD000051F7B2E06B2E712C1A8245C08A81992777
:10FD1000382F22278B819927282B392BF3E06F2E40
:10FD2000712C620E731E1A82AE014D5F5F4FE4317B
:10FD3000B9F4EBBEF60187919691FA018193892F70
:10FD40009927DF018D93AD0182E090E0A0E0B0E063
:10FD5000C80ED91EEA1EFB1E2250304051F713C0B8
:10FD6000CEBABB27AF2D9E2D8D2D8FBB0894C11C05
:10FD7000D11CE11CF11CE09A8DB3DA018D93AD0129
:10FD80002150304069F7FA01108205C092E0692ED7
:10FD9000712C80EC8A838BE10E941AFC0BE1832D8D
:10FDA0000E941AFC0325872D9927182F0E941AFC00
:10FDB0000127862D0E941AFC06258EE00E941AFC5F
:10FDC0008EE008275E010894A11CB11C6114710427
:10FDD00059F0D5011D915D01812F0E941AFC012768
:10FDE000089461087108F2CF802F0E941AFC3394A6
:10FDF0007FCD809164008B7F80936400809165004B
:10FE00008B7F8093650084E690E00E9403FC0000F5
:10FE1000599881E180936800E8951F921F92089598
:02FE2000FFCF12
:040000031000F800F1
:00000001FF
